:100000000C9462000C9481000C9481000C9481008B
:100010000C9481000C9481000C9481000C9481005C
:100020000C9481000C9486080C9481000C9481003F
:100030000C9481000C9481000C9481000C9481003C
:100040000C9481000C9481000C9481000C9481002C
:100050000C9481000C9481000C9481000C9481001C
:100060000C9481000C9481000C9481000C9481000C
:100070000C9481000C9481000C9457020C94810024
:100080000C941A020C942E030C9481000F14141F6C
:1000900014141700010E1315190E1000040A040E93
:1000A000111F110000001A050F140F0000020E1599
:1000B000150E0800040A0E010F110F000C12120C8D
:1000C0000000000011241FBECFEFD0E1DEBFCDBF86
:1000D00011E0A0E0B1E0E6E0F5E100E00BBF02C016
:1000E00007900D92A031B107D9F714E0A0E1B1E07B
:1000F00001C01D92AF35B107E1F70E9484000C9456
:10010000810A0C9400000895EF920F931F93F894C6
:100110000E94EC050E947F080E94CF070E94BE014A
:100120000E942F0681E08093500360E070E080E041
:1001300090E00E94DD0278948FEF809361008093BD
:10014000620092E3E92E02E310E021E040E050E09B
:1001500060E070E081E796E00E943D0486E9E82EC9
:1001600004EF11E021E040E050E060E070E08CEF4F
:1001700095E00E943D0400E117E221E040E050E0FC
:1001800060E070E085E298E00E943D040E9447052F
:10019000FDCFF8942091590430915A0440915B04AA
:1001A00050915C048091540490915504A0915604A0
:1001B000B0915704281739074A075B0760F0789415
:1001C00041E060E171E082E00E94F90289EC90E098
:1001D0000E94CD05089578940895EF920F931F9390
:1001E000DF93CF930F92CDB7DEB79C01FC019081D6
:1001F000923131F480914F048F5F80934F04B3C0EC
:100200009131A1F4D9012EE334E0FD018181F9019E
:100210008083FD018181882309F4A5C011962F5F99
:100220003F4FF4E02E343F0781F79DC0913009F035
:100230009AC08181823139F4909311018093120127
:1002400080914F043DC0883809F03DC09983F894EF
:100250008091590490915A04A0915B04B0915C0480
:100260008093500490935104A0935204B09353048C
:100270007894805D9A48AF4FBF4F80935404909319
:100280005504A0935604B093570441E0BE016F5F3C
:100290007F4F82E00E94F90222E3E22E08EE13E093
:1002A00021E040E050E060E070E089EC90E00E94E6
:1002B0003D0481E08093110188E8809312018FEF63
:1002C000809313014AC08331B9F490931101809354
:1002D0001201F89480915C048093130180915B0477
:1002E0008093140180915A048093150180915904E0
:1002F00080931601789416C08431B9F4909311015B
:1003000080931201809157048093130180915604C9
:1003100080931401809155048093150180915404B9
:100320008093160166E070E01AC0803979F4F89481
:1003300017BE15BC1EBC1FBC2DE088E190E00FB6B7
:10034000F894A89581BD0FBE21BDFFCF90931101F8
:100350008FEF809312011092130163E070E081E14E
:1003600091E00E94CA0180B18095809362000F9055
:10037000CF91DF911F910F91EF9008951092980007
:1003800083E08093990088ED80939A0086E08093C3
:100390009D000895AC0180919B0085FFFCCF709378
:1003A0009C0060932B0210923A03109239036F5F06
:1003B0007F4F70933E0360933D036150704081E036
:1003C00090E090933C0380933B03DA0120E030E01F
:1003D00007C02F5F3F4F8D91F901E55DFD4F808391
:1003E00026173707B0F30895BC0180919B0087FF63
:1003F000FCCF30919C0080919B0087FFFCCF209127
:100400009C00932F80E0AC01420F511D20E030E0B2
:100410000CC080919B0087FFFCCF80919C00FB016A
:10042000E20FF31F80832F5F3F4F2417350788F3B8
:10043000CA0108951F920F920FB60F920BB60F923A
:1004400011242F933F938F939F93EF93FF932091CA
:10045000390330913A0380913D0390913E03281770
:10046000390780F48091390390913A03FC01E55DEE
:10047000FD4F208120939C00019690933A03809336
:10048000390308C010923A031092390310923C03CA
:1004900010923B03FF91EF919F918F913F912F918C
:1004A0000F900BBE0F900FBE0F901F9018951F92CC
:1004B0000F920FB60F920BB60F921124EF920F937B
:1004C0001F932F933F934F935F936F937F938F93DC
:1004D0009F93AF93BF93EF93FF93809129029091E5
:1004E0002A02892B99F481E090E090932A0280936C
:1004F000290220919C00922F80E090932802809303
:100500002702109226021092250241C080912502F6
:1005100090912602892B69F48091270290912802FC
:1005200020919C00820F911D9093280280932702B6
:1005300025C0E0912502F091260280919C00EA5EA0
:10054000FE4F808320912502309126028091270260
:10055000909128022817390788F010922A021092E9
:100560002902EE2400E010E020E047E252E067E1DB
:1005700071E08DEE90E00E94C50409C080912502D3
:100580009091260201969093260280932502FF9176
:10059000EF91BF91AF919F918F917F916F915F91FB
:1005A0004F913F912F911F910F91EF900F900BBEA4
:1005B0000F900FBE0F901F90189580915003880FD9
:1005C00081608093720080E280937000E1E7F0E048
:1005D00080818C7F808385EC8093740081E08093A0
:1005E000400310923F038FEF80934F0310924E030E
:1005F0000895582F80914003813031F1809140035C
:10060000843059F521C08C91F901EF5BFC4F828356
:1006100080914D039D91892780934D032F5F3F4F1C
:100620002617370784F310923F0340934203852F28
:1006300090E0880F991F8093410385EA80937400AE
:1006400082E08093400308958FEF80934D03DB0198
:1006500020E030E0642F70E0E3CF08951F920F9206
:100660000FB60F920BB60F921124EF920F931F93B8
:100670002F933F934F935F936F937F938F939F93AA
:10068000AF93BF93EF93FF9380914003817C09F474
:100690007AC08091710090E0887F907080389105D9
:1006A000A1F0813891054CF48036910509F45AC0C7
:1006B0008037910509F065C055C08039910529F052
:1006C000803A910509F05DC05AC0809140038034A2
:1006D00049F480917300809342038FEF80934F031E
:1006E00080E83DC080914003803809F048C0909177
:1006F0003F03809142039817A0F480913F03E82FB5
:10070000F0E090917300EF5BFC4F92838F5F8093DA
:100710003F0390914F0380917300892780934F038B
:100720002EC08091730080934D0390914F03809170
:100730004D03981711F081E001C082E080934E03D1
:10074000EE2400E010E020E040E050E061E473E0DF
:1007500083E890E00E94C50410923F0381E08093FB
:1007600040030DC0809173008093410310924E03AB
:1007700010923F0385EC8093740080E45FC085ECA9
:1007800064C085E462C08091710090E0887F9070C1
:100790008831910579F08832910599F0089709F030
:1007A00050C0809141038093730085E8809374006A
:1007B00088E044C010923F0380914203809373000D
:1007C00039C090913F0380914203981751F4809172
:1007D0004D038093730080913F038F5F80933F03AD
:1007E00029C020913F038091420330E090E00196C0
:1007F0002817390799F485E98093740080E2809383
:100800004003EE2400E010E020E040E050E060E033
:1008100070E08DED92E00E94C50419C090913F03F5
:10082000E92FF0E0EF5BFC4F8281809373009F5FC4
:1008300090933F0385E88093740080E180934003A8
:1008400006C084E08093400385E080937400FF91AC
:10085000EF91BF91AF919F918F917F916F915F9138
:100860004F913F912F911F910F91EF900F900BBEE1
:100870000F900FBE0F901F901895CF92DF92EF92BE
:10088000FF920F931F93CF93DF936C01F22E9E2D57
:1008900020E030E0A22FF901B4E0EE0FFF1FBA957F
:1008A000E1F7EF5AFC4F8685882331F0AF5F2F5F69
:1008B0003F4F2C30310571F7CA2FD0E0DE0124E024
:1008C000AA0FBB1F2A95E1F7AF5ABC4F1196DC92D5
:1008D000CE92FE0184E0EE0FFF1F8A95E1F7ED5AFC
:1008E000FC4F71836083FE0164E0EE0FFF1F6A9589
:1008F000E1F7EB5AFC4F51834083FD01F6829923C7
:1009000011F4178607C0923311F481E001C082E030
:10091000FD01878734E0CC0FDD1F3A95E1F7DE015A
:10092000AF5ABC4FFD018785282F30E02F5E3B4F2B
:10093000F9018081980FFD0195878F5FF901808310
:10094000FD011087078381E08687F8942091590480
:1009500030915A0440915B0450915C04C801A0E0BE
:10096000B0E0820F931FA41FB51FCF5ADC4F8987B9
:100970009A87AB87BC877894DF91CF911F910F91B5
:10098000FF90EF90DF90CF900895CF92DF92EF929B
:10099000FF920F931F93CF93DF93EC016B01F22E25
:1009A0009E2D20E030E0E22EF901A4E0EE0FFF1FC3
:1009B000AA95E1F7EF5AFC4F8685882331F0E3943E
:1009C0002F5F3F4F2C30310571F76E2D70E0DB014A
:1009D000E4E0AA0FBB1FEA95E1F7AF5ABC4F1196AE
:1009E000DC93CE93FB0134E0EE0FFF1F3A95E1F765
:1009F000ED5AFC4FD182C082FB0124E0EE0FFF1FB5
:100A00002A95E1F7EB5AFC4F51834083ED01FE82BA
:100A1000992311F41F8609C0923321F481E0FD016E
:100A2000878703C082E0ED018F8784E0660F771F20
:100A30008A95E1F76F5A7C4FEB01EF85F0E0EF5EAE
:100A4000FB4F8081980F9D878F5F808318870F836E
:100A500081E08E872091590430915A0440915B04C3
:100A600050915C04C801A0E0B0E0820F931FA41F66
:100A7000B51FFB0181879287A387B487DF91CF9150
:100A80001F910F91FF90EF90DF90CF900895CF933B
:100A9000DF93F8944091590450915A0460915B049B
:100AA00070915C04789410921404809117048F5F05
:100AB0008093170480911704883C49F480911604B0
:100AC0008695809315041092160410921704EFEF88
:100AD000FFEF20E030E0E901A4E0CC0FDD1FAA9594
:100AE000E1F7CF5ADC4F8E85882399F0809114046A
:100AF0008F5F8093140489859A85AB85BC854817E0
:100B000059076A077B0728F08D858F1710F4FD853C
:100B1000E22F2F5F3F4F2C303105E9F6EF3FC9F14F
:100B2000809116048F5F80931604FF27E7FDF095F0
:100B300094E0EE0FFF1F9A95E1F7EF01CF5ADC4FDB
:100B400028813981DF01AB5ABC4F6D917C91ED5A00
:100B5000FC4F80819181F90109958E81882349F4A8
:100B60001E86EF85F0E0EF5EFB4F80818150808331
:100B700010C029853A854B855C858F819885A0E0DA
:100B8000B0E0820F931FA41FB51F89879A87AB8798
:100B9000BC8781E0DF91CF910895AC0120E030E087
:100BA000F901B4E0EE0FFF1FBA95E1F7EF5AFC4FE1
:100BB000808191818417950749F41686E785F0E0D6
:100BC000EF5EFB4F80818150808308952F5F3F4F00
:100BD0002C30310529F7089580E090E0FC0124E0F5
:100BE000EE0FFF1F2A95E1F7EF5AFC4F168601968C
:100BF0008C30910599F7089560E081E00E94CD0660
:100C000060E080E80E94CD0680912904882319F0D5
:100C1000813021F514C08EE394E00E94B00760E0BB
:100C200080EC0E94CD0680E091E00E94B0076091C8
:100C30004F0470E080E090E00E940907089586E08C
:100C400091E00E94B00760E08BE80E94CD066091C1
:100C5000400370E080E090E00E94090708951ABA0E
:100C60000895EF920F931F9380913604813069F4B9
:100C7000EE2400E010E020E040E050E060E070E0B2
:100C80008EE698E00E943D041BC09091350491309F
:100C900049F480912904882319F49093290410C001
:100CA00081500CC080913804813051F48091290426
:100CB000813019F41092290403C08F5F80932904B6
:100CC00082E3E82E00E010E020E040E050E060E049
:100CD00070E08CEF95E00E943D041F910F91EF9022
:100CE0000895EF920F931F93CF93DF93AAE2B4E09E
:100CF000C4E3D4E050E020E030E061E04C91F90141
:100D0000E15DFB4F4083188289B390E0022E02C060
:100D1000959587950A94E2F780FF02C06C9305C011
:100D20001C92413011F4488351E02F5F3F4F1196E0
:100D300021962530310511F7513061F4EE2400E0A1
:100D400010E020E040E050E060E070E081E396E0F9
:100D50000E943D04DF91CF911F910F91EF90089574
:100D600087E084BB8AE780F985BB000090E022E041
:100D7000AA9A9295000000000000000083B3AA9890
:100D800083FD916084FD926085FD946086FD98608E
:100D9000215071F715BA892F08950F931F93CF93A0
:100DA000DF93182F062F15BA80913904882361F13B
:100DB000E894C0E0D0E00E94B00687FF21C02196F1
:100DC00083E0C83ED807B9F7109239048FE784BB97
:100DD00022E0802F011181E0912F14FD886095FDA4
:100DE000806196FD806217FD806485BB0000AA9A31
:100DF000129500000000000085BB215051F704C08F
:100E0000C85ED3401CF3E0CFDF91CF911F910F91CB
:100E100008959F92AF92BF92CF92DF92EF92FF928E
:100E20000F931F93CF93DF937B018C0197FF0BC030
:100E300010950095F094E094E11CF11C011D111D2A
:100E400061E08DE207C0611571058105910521F40E
:100E500061E080E30E94CD06A12C8AECB82E8AE9DD
:100E6000C82E8BE3D82E9924CAE0D0E0C801B70180
:100E7000A60195010E94660A992011F4222391F09F
:100E800061E0822F805D0E94CD06C801B701A601F6
:100E900095010E94660AAC01CB01DA017C018D014B
:100EA00099249A94C601B5012AE030E040E050E070
:100EB0000E94660AC901DA015C016D012197B1F651
:100EC000DF91CF911F910F91FF90EF90DF90CF9026
:100ED000BF90AF909F900895AF92BF92CF92DF9254
:100EE000EF92FF920F931F937B018C015A01CC2448
:100EF000DD24C601B5010E9453099B01AC01C80164
:100F0000B7010E94E1090E9422097B018C01C801FE
:100F1000A60195010E94660ACA01B9010E9409074B
:100F200061E08EE20E94CD06B701C801A6019501DD
:100F30000E94660A0E9455099F7720E030E040E059
:100F40005FE30E94BE080E9422090E9409071F91C8
:100F50000F91FF90EF90DF90CF90BF90AF900895EA
:100F6000CF93DF93EC0104C0219661E00E94CD068F
:100F700088818823C9F7DF91CF910895CF93DF93BC
:100F8000FC01EC01849105C061E00E94CD06FE01E8
:100F9000849121968823C1F7DF91CF9108950F9313
:100FA0001F9381E0809339048FE784BB4FE024E0F6
:100FB00030E06FEF7FE350E1CB010197F1F741FBA8
:100FC00083F985BB0000AA9A000000000000000021
:100FD000AA9846952150304079F760E088E20E9457
:100FE000CD0680913904882319F160E086E00E94E3
:100FF000CD0660E082E00E94CD0660E08CE00E94B9
:10100000CD0660E088E40E94CD06ECE8F0E008C080
:101010008F010F5F1F4F849161E00E94CD06F801A0
:1010200080E0E43CF807A0F360E080E80E94CD0691
:1010300080E01F910F910895E8940E94B00660E04F
:1010400080680E94CD0680E00895DF93CF9300D0A2
:1010500000D00F92CDB7DEB72091540430915504E3
:101060004091560450915704211531054105510511
:10107000B9F0F8946091590470915A0480915B041E
:1010800090915C04621B730B840B950B789420E6A3
:101090003AEE40E050E00E94440A3A83298304C0BB
:1010A0008FEF9FEF9A838983FE01339683E0DF0100
:1010B0001D928A95E9F785E18B8389818C838A81EA
:1010C0008D8363E070E0CF010E94CA010F900F9002
:1010D0000F900F900F90CF91DF910895DF93CF93F2
:1010E0000F92CDB7DEB784E3898361E070E0CE0173
:1010F00001960E94CA010F90CF91DF9108958BE075
:1011000085BD89EF83BD80E887BF08951F920F9248
:101110000FB60F9211248F939F93AF93BF9380913B
:10112000590490915A04A0915B04B0915C0401961B
:10113000A11DB11D8093590490935A04A0935B04A0
:10114000B0935C04809158048F5F809358048A3078
:1011500059F41092580480915D0490915E040196B8
:1011600090935E0480935D04BF91AF919F918F91A6
:101170000F900FBE0F901F9018955058BB27AA27AD
:101180000ED0E5C0D6D030F0DBD020F031F49F3F58
:1011900011F41EF4CBC00EF4E095E7FBC1C0E92FBB
:1011A000E7D080F3BA17620773078407950718F032
:1011B00071F49EF5FFC00EF4E0950B2EBA2FA02D12
:1011C0000B01B90190010C01CA01A0011124FF27F4
:1011D000591B99F0593F50F4503E68F11A16F040EF
:1011E000A22F232F342F4427585FF3CF46953795EE
:1011F0002795A795F0405395C9F77EF41F16BA0BB3
:10120000620B730B840BBAF09150A1F0FF0FBB1F60
:10121000661F771F881FC2F70EC0BA0F621F731FA9
:10122000841F48F4879577956795B795F7959E3F06
:1012300008F0B3CF9395880F08F09927EE0F979594
:101240008795089504D06894B111B5C0089598D0D9
:1012500088F09F5790F0B92F9927B751A0F0D1F09F
:10126000660F771F881F991F1AF0BA95C9F712C029
:10127000B13081F09FD0B1E008959CC0672F782FE6
:101280008827B85F39F0B93FCCF386957795679595
:10129000B395D9F73EF490958095709561957F4F01
:1012A0008F4F9F4F0895E89409C097FB3EF49095A7
:1012B0008095709561957F4F8F4F9F4F9923A9F02F
:1012C000F92F96E9BB279395F695879577956795BE
:1012D000B795F111F8CFFAF4BB0F11F460FF1BC002
:1012E0006F5F7F4F8F4F9F4F16C0882311F096E995
:1012F00011C0772321F09EE8872F762F05C0662343
:1013000071F096E8862F70E060E02AF09A95660FFB
:10131000771F881FDAF7880F9695879597F90895B4
:1013200097F99F6780E870E060E008959FEF80EC98
:10133000089500240A94161617061806090608953B
:1013400000240A9412161306140605060895092EA1
:101350000394000C11F4882352F0BB0F40F4BF2B10
:1013600011F460FF04C06F5F7F4F8F4F9F4F089550
:1013700057FD9058440F551F59F05F3F71F0479546
:10138000880F97FB991F61F09F3F79F0879508952B
:10139000121613061406551FF2CF4695F1DF08C04A
:1013A000161617061806991FF1CF86957105610567
:1013B00008940895E894BB2766277727CB0197F90F
:1013C00008950BD0C4CFB5DF28F0BADF18F095230D
:1013D00009F0A6CFABCF1124EECFCADFA0F3959FC3
:1013E000D1F3950F50E0551F629FF001729FBB270C
:1013F000F00DB11D639FAA27F00DB11DAA1F649FB8
:101400006627B00DA11D661F829F2227B00DA11D6A
:10141000621F739FB00DA11D621F839FA00D611DF0
:10142000221F749F3327A00D611D231F849F600D11
:10143000211D822F762F6A2F11249F5750408AF04A
:10144000E1F088234AF0EE0FFF1FBB1F661F771FD6
:10145000881F91505040A9F79E3F510570F060CF12
:10146000AACF5F3FECF3983EDCF3869577956795BE
:10147000B795F795E7959F5FC1F7FE2B880F911DF4
:101480009695879597F90895A1E21A2EAA1BBB1B82
:10149000FD010DC0AA1FBB1FEE1FFF1FA217B30740
:1014A000E407F50720F0A21BB30BE40BF50B661F56
:1014B000771F881F991F1A9469F76095709580951A
:1014C00090959B01AC01BD01CF01089597FB092EBA
:1014D00005260ED057FD04D0D7DF0AD0001C38F403
:1014E00050954095309521953F4F4F4F5F4F089550
:1014F000F6F790958095709561957F4F8F4F9F4F30
:061500000895F894FFCFEE
:10150600486974733A0054776920737461743A00B9
:020000021000EC
:10E000000C9446F00C9465F00C9465F00C9465F05B
:10E010000C9465F00C9465F00C9465F00C9465F02C
:10E020000C9465F00C9465F00C9465F00C9465F01C
:10E030000C9465F00C9465F00C9465F00C9465F00C
:10E040000C9465F00C9465F00C9465F00C9465F0FC
:10E050000C9465F00C9465F00C9465F00C9465F0EC
:10E060000C9465F00C9465F00C9465F00C9465F0DC
:10E070000C9465F00C9465F00C9465F00C9465F0CC
:10E080000C9465F00C9465F00C9465F011241FBE9F
:10E09000CFEFD0E1DEBFCDBF11E0A0E0B1E0E2E61E
:10E0A000F4EE01E00BBF02C007900D92A030B10763
:10E0B000D9F711E0A0E0B1E001C01D92A030B10796
:10E0C000E1F70E945BF10C942FF20C9400F008959C
:10E0D000CF93DF93EC0185E08EBD86B7846086BF69
:10E0E00080919B0087FD03C006B602FEF9CF06B6FD
:10E0F00002FE09C085B7816085BF85B78D7F85BF6A
:10E10000E0E0F0E009951EBC30919C0080919B00FE
:10E1100087FFFCCF20919C00932F80E0AC01420F41
:10E12000511D20E030E00CC080919B0087FFFCCFA8
:10E1300080919C00FE01E20FF31F80832F5F3F4F11
:10E140002417350788F3CA01DF91CF910895BC01E8
:10E1500080919B0087FFFCCF30919C0080919B00B9
:10E1600087FFFCCF20919C00932F80E0AC01420FF1
:10E17000511D20E030E00CC080919B0087FFFCCF58
:10E1800080919C00FB01E20FF31F80832F5F3F4FC4
:10E190002417350788F3CA010895AC0180919B00CC
:10E1A00085FFFCCF70939C0080919B0085FFFCCF86
:10E1B00060939C0020E030E00CC080919B0085FFC4
:10E1C000FCCFFA01E20FF31F808180939C002F5F48
:10E1D0003F4F2617370788F308951092980083E081
:10E1E00080939900EBE9F0E080818D7F808388E166
:10E1F00080939A0086E080939D000895BF92CF920D
:10E20000DF92EF92FF920F931F93CF93DF937B01E7
:10E210008C016A01E199FECF83E0F70100935B0076
:10E2200080936800E8958091680080FDFCCF40E015
:10E2300050E060E070E0BB24B394F6018081D181AE
:10E24000C0E09E01280F311D82E090E0C80ED91E6B
:10E25000DB01CA018E0D9F1DA01FB11F0901FC012A
:10E26000A0935B00B0926800E89511244E5F5F4F69
:10E270006F4F7F4F403091E0590790E0690790E081
:10E280007907D9F685E0F70100935B008093680079
:10E29000E8958091680080FDFCCF81E18093680063
:10E2A000E895DF91CF911F910F91FF90EF90DF9054
:10E2B000CF90BF90089524B714BE88E10FB6F894AC
:10E2C00081BD11BC0FBE1124D2E0C0E0F89485B727
:10E2D000816085BF85B7826085BF8FEF90E19EBF6B
:10E2E0008DBF1092980083E08093990080919B00ED
:10E2F0008D7F80939B0088E180939A0086E08093D5
:10E300009D0023FF0AC081E0898382E98A8362E05D
:10E3100070E0CE0101960E94CDF08E010A5F1F4F82
:10E32000C8010E9468F08D8590E0A0E0B0E07C011B
:10E33000DD24CC248E8590E0A0E0B0E0BA2FA92F98
:10E34000982F8827C80ED91EEA1EFB1E8F85C80E7F
:10E35000D11CE11CF11C81E0898381E98A8344247A
:10E36000552488249924540122242A945DC03B8298
:10E370004C8264E070E0CE0101960E94CDF0809165
:10E380009B0087FFFCCF90919C0080919B0087FFB2
:10E39000FCCF80919C00792E66248301080F111D0B
:10E3A00020E030E00FC080919B0087FFFCCF809180
:10E3B0009C00E6E0F0E0EC0FFD1FE20FF31F80830E
:10E3C0002F5F3F4F2017310770F38E81813079F630
:10E3D0008F81813949F599858B81981729F59A851F
:10E3E0008C81981709F5E6E0F0E0EC0FFD1FE00FD7
:10E3F000F11FC80102C02192019621E085309207E9
:10E40000D0F3AE01455F5F4FC501B4010E94FEF03D
:10E4100005501040C801A0E0B0E0880E991EAA1E69
:10E42000BB1E0894411C511C8C149D04AE04BF04F7
:10E4300010F4352C9CCF80E98A8362E070E0CE0135
:10E4400001960E94CDF01EBC85B7816085BF85B75F
:10E450008D7F85BFE0E0F0E0099580E090E0F894E2
:02E46000FFCFEC
:040000031000E00009
:00000001FF
